 srvclum

 Timestamp is 4be8c237 (Tue May 11 11:34:31 2010)

 Preferred load address is 10000000

 Start         Length     Name                   Class
 0001:00000000 00000004H .CRT$XCA                CODE
 0001:00000004 00000004H .CRT$XCZ                CODE
 0001:00000008 00000004H .CRT$XIA                CODE
 0001:0000000c 00000004H .CRT$XIZ                CODE
 0001:00000010 00000004H .CRT$XPA                CODE
 0001:00000014 00000004H .CRT$XPZ                CODE
 0001:00000018 00000004H .CRT$XTA                CODE
 0001:0000001c 00000004H .CRT$XTZ                CODE
 0001:00000020 000012c4H .rdata                  CODE
 0001:000012e4 00000024H .rdata$debug            CODE
 0001:00001308 0000f54cH .text                   CODE
 0001:00010854 00000044H .xdata                  CODE
 0001:00010898 00000014H .idata$2                CODE
 0001:000108ac 00000014H .idata$3                CODE
 0001:000108c0 000000c4H .idata$4                CODE
 0001:00010984 0000000cH .idata$6                CODE
 0001:00010990 000009f4H .edata                  CODE
 0002:00000000 000000c4H .idata$5                DATA
 0002:000000c8 000005f0H .data                   DATA
 0002:000006b8 00000418H .bss                    DATA
 0003:00000000 00000630H .pdata                  DATA

  Address         Publics by Value              Rva+Base       Lib:Object

 0000:00000000       ___safe_se_handler_table   00000000     <absolute>
 0000:00000000       ___safe_se_handler_count   00000000     <absolute>
 0001:00000000       __xc_a                     10001000     corelib0:crt0init.obj
 0001:00000004       __xc_z                     10001004     corelib0:crt0init.obj
 0001:00000008       __xi_a                     10001008     corelib0:crt0init.obj
 0001:0000000c       __xi_z                     1000100c     corelib0:crt0init.obj
 0001:00000010       __xp_a                     10001010     corelib0:crt0init.obj
 0001:00000014       __xp_z                     10001014     corelib0:crt0init.obj
 0001:00000018       __xt_a                     10001018     corelib0:crt0init.obj
 0001:0000001c       __xt_z                     1000101c     corelib0:crt0init.obj
 0001:00000388       ??_C@_15MAOEGKJF@?$AA?$CF?$AAS?$AA?$AA@ 10001388     srvclient_wince.obj
 0001:00000390       ??_C@_09PDOEPFPA@?$FLdefault?$FN?$AA@ 10001390     pvr_apphint.obj
 0001:0000039c       ??_C@_04LIFAFMCE@?$FL?$CFs?$FN?$AA@ 1000139c     pvr_apphint.obj
 0001:000003a4       ??_C@_01KDCPPGHE@r?$AA@    100013a4     pvr_apphint.obj
 0001:000003a8       ??_C@_0M@IIKDEAIO@powervr?4ini?$AA@ 100013a8     pvr_apphint.obj
 0001:000003b4       ??_C@_0BF@HAPGGGPH@?2windows?2powervr?4ini?$AA@ 100013b4     pvr_apphint.obj
 0001:000003cc       ??_C@_1M@DMCDIEDK@?$AAP?$AAK?$AAM?$AA1?$AA?3?$AA?$AA@ 100013cc     srvclientenvumcmn:pvr_bridge_u.obj
 0001:000003d8       ??_C@_09KIHBNIPC@?5?$CI?$CFu?0?$CFs?$CJ?6?$AA@ 100013d8     srvclientenvumcmn:pvr_debug.obj
 0001:000003e4       ??_C@_05CIJMOPAN@PVR?3?5?$AA@ 100013e4     srvclientenvumcmn:pvr_debug.obj
 0001:000003ec       ??_C@_0BI@NLGOAFIB@Debug?5assertion?5failed?$CB?$AA@ 100013ec     srvclientenvumcmn:pvr_debug.obj
 0001:00000404       ??_C@_01EEMJAFIK@?6?$AA@   10001404     srvclientenvumcmn:pvr_debug.obj
 0001:00000408       ??_C@_0BF@JAPCMFOG@MTModePixelThreshold?$AA@ 10001408     srvclientsgx:sgxrender_targets.obj
 0001:00000588       ??_C@_0N@EMGKHBNG@PDSThreshold?$AA@ 10001588     srvclientsgx:sgxrender_context.obj
 0001:00000598       ??_C@_0BA@PNIFOOAA@GlobalThreshold?$AA@ 10001598     srvclientsgx:sgxrender_context.obj
 0001:000005a8       ??_C@_0N@HADJGBAO@ZLSThreshold?$AA@ 100015a8     srvclientsgx:sgxrender_context.obj
 0001:000005b8       ??_C@_0M@MLMDFGLM@TAThreshold?$AA@ 100015b8     srvclientsgx:sgxrender_context.obj
 0001:000005c4       ??_C@_0BB@PPHBJPP@EDMProtectTATest?$AA@ 100015c4     srvclientsgx:sgxrender_context.obj
 0001:000005d8       ??_C@_0BD@CEJJAMAG@NumPixelPartitions?$AA@ 100015d8     srvclientsgx:sgxrender_context.obj
 0001:000005ec       ??_C@_0BE@MDMDMIME@NumVertexPartitions?$AA@ 100015ec     srvclientsgx:sgxrender_context.obj
 0001:00000600       ??_C@_06HLKHBNKH@PBSize?$AA@ 10001600     srvclientsgx:sgxrender_context.obj
 0001:00000608       ??_C@_0BD@JBLBCAKP@UseSharedParamHeap?$AA@ 10001608     srvclientsgx:sgxrender_context.obj
 0001:00001308       PDSGeneratePixelEventProgram 10002308 f   pds.obj
 0001:000013a8       WriteEndOfRenderUSSECode   100023a8 f   pixevent.obj
 0001:000013d8       WriteEndOfTileUSSECode     100023d8 f   pixevent.obj
 0001:00001498       SGXFindSharedPBDesc        10002498 f   bridged_sgx_glue.obj
 0001:000015bc       SGXUnrefSharedPBDesc       100025bc f   bridged_sgx_glue.obj
 0001:00001628       SGXAddSharedPBDesc         10002628 f   bridged_sgx_glue.obj
 0001:000016dc       SGXSubmitTransferBridge    100026dc f   bridged_sgx_glue.obj
 0001:00001754       SGXRegisterHWRenderContext 10002754 f   bridged_sgx_glue.obj
 0001:000017e8       SGXUnregisterHWRenderContext 100027e8 f   bridged_sgx_glue.obj
 0001:00001858       SGXRegisterHWTransferContext 10002858 f   bridged_sgx_glue.obj
 0001:000018ec       SGXUnregisterHWTransferContext 100028ec f   bridged_sgx_glue.obj
 0001:00001960       SGXFlushHWRenderTarget     10002960 f   bridged_sgx_glue.obj
 0001:000019d4       SGXDoKick                  100029d4 f   bridged_sgx_glue.obj
 0001:00001a6c       SGXGetClientInfo           10002a6c f   bridged_sgx_glue.obj
 0001:00001b88       SGXReleaseClientInfo       10002b88 f   bridged_sgx_glue.obj
 0001:00001c40       SGXGetInternalDevInfo      10002c40 f   bridged_sgx_glue.obj
 0001:00001ce8       SGXGetMiscInfo             10002ce8 f   bridged_sgx_glue.obj
 0001:00001d4c       SGX2DQueryBlitsComplete    10002d4c f   bridged_sgx_glue.obj
 0001:00001dc8       PVRSRVEnumerateDeviceClass 10002dc8 f   bridged_pvr_glue.obj
 0001:00001e8c       PVRSRVConnect              10002e8c f   bridged_pvr_glue.obj
 0001:00001ebc       PVRSRVDisconnect           10002ebc f   bridged_pvr_glue.obj
 0001:00001ec4       PVRSRVEnumerateDevices     10002ec4 f   bridged_pvr_glue.obj
 0001:00001f70       PVRSRVAcquireDeviceData    10002f70 f   bridged_pvr_glue.obj
 0001:00001ff4       PVRSRVCreateDeviceMemContext 10002ff4 f   bridged_pvr_glue.obj
 0001:000020cc       PVRSRVDestroyDeviceMemContext 100030cc f   bridged_pvr_glue.obj
 0001:00002140       PVRSRVGetDeviceMemHeapInfo 10003140 f   bridged_pvr_glue.obj
 0001:00002214       PVRSRVExportDeviceMem      10003214 f   bridged_pvr_glue.obj
 0001:000022a8       PVRSRVWrapExtMemory        100032a8 f   bridged_pvr_glue.obj
 0001:000024ac       PVRSRVUnwrapExtMemory      100034ac f   bridged_pvr_glue.obj
 0001:00002560       PVRSRVMapDeviceClassMemory 10003560 f   bridged_pvr_glue.obj
 0001:000026c4       PVRSRVUnmapDeviceClassMemory 100036c4 f   bridged_pvr_glue.obj
 0001:00002774       PVRSRVGetMiscInfo          10003774 f   bridged_pvr_glue.obj
 0001:00002854       PVRSRVMapPhysToUserSpace   10003854 f   bridged_pvr_glue.obj
 0001:000028e4       PVRSRVUnmapPhysToUserSpace 100038e4 f   bridged_pvr_glue.obj
 0001:0000293c       PVRSRVGetMMUContextPDDevPAddr 1000393c f   bridged_pvr_glue.obj
 0001:00002998       PVRSRVUnmapDeviceMemory    10003998 f   bridged_pvr_glue.obj
 0001:00002a30       PVRSRVOpenBCDevice         10003a30 f   bridged_pvr_bc_glue.obj
 0001:00002ac0       PVRSRVCloseBCDevice        10003ac0 f   bridged_pvr_bc_glue.obj
 0001:00002b3c       PVRSRVGetBCBufferInfo      10003b3c f   bridged_pvr_bc_glue.obj
 0001:00002bc4       PVRSRVGetBCBuffer          10003bc4 f   bridged_pvr_bc_glue.obj
 0001:00002c58       PVRSRVOpenDCDevice         10003c58 f   bridged_pvr_dc_glue.obj
 0001:00002ce8       PVRSRVCloseDCDevice        10003ce8 f   bridged_pvr_dc_glue.obj
 0001:00002d70       PVRSRVEnumDCFormats        10003d70 f   bridged_pvr_dc_glue.obj
 0001:00002e3c       PVRSRVEnumDCDims           10003e3c f   bridged_pvr_dc_glue.obj
 0001:00002f18       PVRSRVGetDCSystemBuffer    10003f18 f   bridged_pvr_dc_glue.obj
 0001:00002fa8       PVRSRVGetDCInfo            10003fa8 f   bridged_pvr_dc_glue.obj
 0001:0000306c       PVRSRVCreateDCSwapChain    1000406c f   bridged_pvr_dc_glue.obj
 0001:00003198       PVRSRVDestroyDCSwapChain   10004198 f   bridged_pvr_dc_glue.obj
 0001:00003208       PVRSRVSetDCDstRect         10004208 f   bridged_pvr_dc_glue.obj
 0001:000032a4       PVRSRVGetDCBuffers         100042a4 f   bridged_pvr_dc_glue.obj
 0001:00003358       PVRSRVSwapToDCBuffer       10004358 f   bridged_pvr_dc_glue.obj
 0001:0000343c       PVRSRVSwapToDCSystem       1000443c f   bridged_pvr_dc_glue.obj
 0001:000034b0       PVRPMapKMem                100044b0 f   srvclient_wince.obj
 0001:000034b8       PVRUnMapKMem               100044b8 f   srvclient_wince.obj
 0001:000034c8       PVRSRVEventObjectOpen      100044c8 f   srvclient_wince.obj
 0001:00003530       PVRSRVEventObjectClose     10004530 f   srvclient_wince.obj
 0001:00003538       PVRSRVEventObjectWait      10004538 f   srvclient_wince.obj
 0001:00003578       PVRSRVUnlockResource       10004578 f   srvclient_wince.obj
 0001:000035ac       PVRSRVCallocUserModeMem    100045ac f   srvclient_wince.obj
 0001:000035b8       PVRSRVReallocUserModeMem   100045b8 f   srvclient_wince.obj
 0001:000035bc       PVRSRVClockus              100045bc f   srvclient_wince.obj
 0001:000035d4       PVRSRVWaitus               100045d4 f   srvclient_wince.obj
 0001:00003614       PVRSRVMemCopy              10004614 f   srvclient_wince.obj
 0001:00003618       PVRSRVMemSet               10004618 f   srvclient_wince.obj
 0001:0000361c       PVRSRVCreateMutex          1000461c f   srvclient_wince.obj
 0001:00003644       PVRSRVDestroyMutex         10004644 f   srvclient_wince.obj
 0001:00003654       PVRSRVUnlockMutex          10004654 f   srvclient_wince.obj
 0001:00003674       PVRSRVLockResource         10004674 f   srvclient_wince.obj
 0001:000036d4       PVRSRVLockMutex            100046d4 f   srvclient_wince.obj
 0001:000037c0       FindAppHintInFile          100047c0 f   pvr_apphint.obj
 0001:000039cc       FindAppHint                100049cc f   pvr_apphint.obj
 0001:00003a64       PVRSRVCreateAppHintState   10004a64 f   pvr_apphint.obj
 0001:00003a90       PVRSRVFreeAppHintState     10004a90 f   pvr_apphint.obj
 0001:00003aa4       PVRSRVGetAppHint           10004aa4 f   pvr_apphint.obj
 0001:00003b20       PVRSRVAllocUserModeMem     10004b20 f   srvclientenvumcmn:osfunc_umclient.obj
 0001:00003b24       PVRSRVFreeUserModeMem      10004b24 f   srvclientenvumcmn:osfunc_umclient.obj
 0001:00003b28       PVRSRVReleaseThreadQuanta  10004b28 f   srvclientenvumcmn:osfunc_umclient.obj
 0001:00003b30       PVRSRVGetCurrentProcessID  10004b30 f   srvclientenvumcmn:osfunc_umclient.obj
 0001:00003b38       PVRSRVSetLocale            10004b38 f   srvclientenvumcmn:osfunc_umclient.obj
 0001:00003b48       PVRSRVLoadLibrary          10004b48 f   srvclientenvumcmn:osfunc_umclient.obj
 0001:00003bc0       PVRSRVUnloadLibrary        10004bc0 f   srvclientenvumcmn:osfunc_umclient.obj
 0001:00003be0       PVRSRVGetLibFuncAddr       10004be0 f   srvclientenvumcmn:osfunc_umclient.obj
 0001:00003c80       OSIsProcessPrivileged      10004c80 f   srvclientenvumcmn:osfunc_umclient.obj
 0001:00003c88       PVRSRVBridgeCall           10004c88 f   srvclientenvumcmn:pvr_bridge_u.obj
 0001:00003d34       OpenServices               10004d34 f   srvclientenvumcmn:pvr_bridge_u.obj
 0001:00003dec       CloseServices              10004dec f   srvclientenvumcmn:pvr_bridge_u.obj
 0001:00003e58       PVRSRVReleaseMiscInfo      10004e58 f   srvclientenvumcmn:pvr_glue.obj
 0001:00003f24       PVRSRVAllocDeviceMem       10004f24 f   srvclientenvumcmn:pvr_glue.obj
 0001:00004058       PVRSRVFreeDeviceMem        10005058 f   srvclientenvumcmn:pvr_glue.obj
 0001:000041c4       PVRSRVUnrefDeviceMem       100051c4 f   srvclientenvumcmn:pvr_glue.obj
 0001:000041c8       PVRSRVMapDeviceMemory      100051c8 f   srvclientenvumcmn:pvr_glue.obj
 0001:00004358       PVRSRVFreeSharedSysMem     10005358 f   srvclientenvumcmn:pvr_glue.obj
 0001:000043e0       PVRSRVUnrefSharedSysMem    100053e0 f   srvclientenvumcmn:pvr_glue.obj
 0001:000043e4       PVRSRVAllocSharedSysMem    100053e4 f   srvclientenvumcmn:pvr_glue.obj
 0001:000044d8       PVRSRVMapMemInfoMem        100054d8 f   srvclientenvumcmn:pvr_glue.obj
 0001:000045e0       PVRSRVAllocUserModeMemTracking 100055e0 f   srvclientenvumcmn:memchk.obj
 0001:000045e8       PVRSRVCallocUserModeMemTracking 100055e8 f   srvclientenvumcmn:memchk.obj
 0001:000045f0       PVRSRVFreeUserModeMemTracking 100055f0 f   srvclientenvumcmn:memchk.obj
 0001:000045f4       PVRSRVReallocUserModeMemTracking 100055f4 f   srvclientenvumcmn:memchk.obj
 0001:00004604       PVRSRVDebugPrintf          10005604 f   srvclientenvumcmn:pvr_debug.obj
 0001:0000472c       PVRSRVDebugAssertFail      1000572c f   srvclientenvumcmn:pvr_debug.obj
 0001:0000474c       PVRSRVTrace                1000574c f   srvclientenvumcmn:pvr_debug.obj
 0001:000053ec       SGXRemoveRenderTarget      100063ec f   srvclientsgx:sgxrender_targets.obj
 0001:00005490       SGXAddRenderTarget         10006490 f   srvclientsgx:sgxrender_targets.obj
 0001:00005f14       SGXDestroyRenderContext    10006f14 f   srvclientsgx:sgxrender_context.obj
 0001:00006348       SGXCreateRenderContext     10007348 f   srvclientsgx:sgxrender_context.obj
 0001:000074ac       SGXDestroyTransferContext  100084ac f   srvclientsgx:sgxtransfer_context.obj
 0001:00007724       SGXCreateTransferContext   10008724 f   srvclientsgx:sgxtransfer_context.obj
 0001:000084e0       SGXKickTA                  100094e0 f   srvclientsgx:sgxkick_client.obj
 0001:0000d3c0       SGXQueueTransfer           1000e3c0 f   srvclientsgx:sgxtransfer_queue.obj
 0001:0000d790       CreateCCB                  1000e790 f   srvclientsgx:sgxutils_client.obj
 0001:0000d8e4       DestroyCCB                 1000e8e4 f   srvclientsgx:sgxutils_client.obj
 0001:0000d910       SGXSetContextPriority      1000e910 f   srvclientsgx:sgxutils_client.obj
 0001:0000da60       SGXTQ_FixedIntDiv          1000ea60 f   srvclientsgx:sgxtransfer_utils.obj
 0001:0000da9c       SGXTQ_FixedToFloat         1000ea9c f   srvclientsgx:sgxtransfer_utils.obj
 0001:0000db1c       SGXTQ_FixedToF16           1000eb1c f   srvclientsgx:sgxtransfer_utils.obj
 0001:0000db9c       SGXTQ_GetTAGFormat         1000eb9c f   srvclientsgx:sgxtransfer_utils.obj
 0001:0000ddcc       SGXTQ_GetPBEFormat         1000edcc f   srvclientsgx:sgxtransfer_utils.obj
 0001:0000df98       SGXTQ_FilterFromEnum       1000ef98 f   srvclientsgx:sgxtransfer_utils.obj
 0001:0000dfc8       SGXTQ_RotationFromEnum     1000efc8 f   srvclientsgx:sgxtransfer_utils.obj
 0001:0000e008       SGXTQ_MemLayoutFromEnum    1000f008 f   srvclientsgx:sgxtransfer_utils.obj
 0001:0000e0dc       SGXTQ_ShaderFromAlpha      1000f0dc f   srvclientsgx:sgxtransfer_utils.obj
 0001:0000e134       SGXTQ_ShaderFromRop        1000f134 f   srvclientsgx:sgxtransfer_utils.obj
 0001:0000e258       SGXTQ_WriteUSEMovToReg     1000f258 f   srvclientsgx:sgxtransfer_utils.obj
 0001:0000e300       SGXTQ_GetStrideGran        1000f300 f   srvclientsgx:sgxtransfer_utils.obj
 0001:0000e32c       SGXTQ_GetSurfaceStride     1000f32c f   srvclientsgx:sgxtransfer_utils.obj
 0001:0000e49c       SGXTQ_GetSurfaceWidth      1000f49c f   srvclientsgx:sgxtransfer_utils.obj
 0001:0000e58c       SGXTQ_SetTAGState          1000f58c f   srvclientsgx:sgxtransfer_utils.obj
 0001:0000e720       SGXTQ_SetUSSEKick          1000f720 f   srvclientsgx:sgxtransfer_utils.obj
 0001:0000e770       SGXTQ_SetDMAState          1000f770 f   srvclientsgx:sgxtransfer_utils.obj
 0001:0000e7b8       SGXTQ_SetupStridedBlit     1000f7b8 f   srvclientsgx:sgxtransfer_utils.obj
 0001:0000e9a8       SGXTQ_SetPBEState          1000f9a8 f   srvclientsgx:sgxtransfer_utils.obj
 0001:0000eae0       SGXTQ_UpdateTileEvent      1000fae0 f   srvclientsgx:sgxtransfer_utils.obj
 0001:0000ec18       SGXTQ_UpdateSecondaryPDSProgramBasic 1000fc18 f   srvclientsgx:sgxtransfer_utils.obj
 0001:0000ec90       SGXTQ_UpdateSecondaryPDSProgram1Attr 1000fc90 f   srvclientsgx:sgxtransfer_utils.obj
 0001:0000ed28       SGXTQ_UpdateSecondaryPDSProgram3Attr 1000fd28 f   srvclientsgx:sgxtransfer_utils.obj
 0001:0000ee00       SGXTQ_UpdateSecondaryPDSProgram4AttrDMA 1000fe00 f   srvclientsgx:sgxtransfer_utils.obj
 0001:0000ef38       SGXTQ_UpdateSecondaryPDSProgramTexSetup 1000ff38 f   srvclientsgx:sgxtransfer_utils.obj
 0001:0000ef4c       SGXTQ_SetupTransferRegs    1000ff4c f   srvclientsgx:sgxtransfer_utils.obj
 0001:0000f044       SGXTQ_UpdatePrimaryPDSSingleSource 10010044 f   srvclientsgx:sgxtransfer_utils.obj
 0001:0000f13c       SGXTQ_UpdatePrimaryPDSTwoSource 1001013c f   srvclientsgx:sgxtransfer_utils.obj
 0001:0000f2b4       SGXTQ_UpdatePrimaryPDSThreeSource 100102b4 f   srvclientsgx:sgxtransfer_utils.obj
 0001:0000f4ac       SGXTQ_UpdatePrimaryPDSIter 100104ac f   srvclientsgx:sgxtransfer_utils.obj
 0001:0000f544       SGXTQ_UpdatePrimaryPDSKickOnly 10010544 f   srvclientsgx:sgxtransfer_utils.obj
 0001:0000f5bc       SGXTQ_SetupTransferRenderBox 100105bc f   srvclientsgx:sgxtransfer_utils.obj
 0001:0000f5f8       SGXTQ_SetupTransferClipRenderBox 100105f8 f   srvclientsgx:sgxtransfer_utils.obj
 0001:0000f668       SGXTQ_UpdateControlObject  10010668 f   srvclientsgx:sgxtransfer_utils.obj
 0001:0000fb2c       SGXTQ_UpdateISPControlStream 10010b2c f   srvclientsgx:sgxtransfer_utils.obj
 0001:0000ff10       SGXTQ_StagingBufferAcquireSpace 10010f10 f   srvclientsgx:sgxtransfer_utils.obj
 0001:0000ffec       SGXTQ_GetStagingBufferDevVAddr 10010fec f   srvclientsgx:sgxtransfer_utils.obj
 0001:0000fffc       SGXTQ_UpdateStagingBuffer  10010ffc f   srvclientsgx:sgxtransfer_utils.obj
 0001:00010018       SGXTQ_ClampInputRects      10011018 f   srvclientsgx:sgxtransfer_utils.obj
 0001:00010098       SGXTQ_CopyToStagingBuffer  10011098 f   srvclientsgx:sgxtransfer_utils.obj
 0001:000100f0       SGXTQ_FloatIntDiv          100110f0 f   srvclientsgx:sgxtransfer_utils.obj
 0001:00010110       PVRSRVPollForValue         10011110 f   srvclientcmn:resources.obj
 0001:000101c8       __GetUserKData             100111c8 f   coredll:COREDLL.dll
 0001:000101d8       CreateEventW               100111d8 f   coredll:COREDLL.dll
 0001:000101e8       WaitForSingleObject        100111e8 f   coredll:COREDLL.dll
 0001:000101f8       GetTickCount               100111f8 f   coredll:COREDLL.dll
 0001:00010208       InterlockedCompareExchange 10011208 f   coredll:COREDLL.dll
 0001:00010218       WideCharToMultiByte        10011218 f   coredll:COREDLL.dll
 0001:00010228       GetModuleFileNameW         10011228 f   coredll:COREDLL.dll
 0001:00010238       Sleep                      10011238 f   coredll:COREDLL.dll
 0001:00010248       LoadLibraryW               10011248 f   coredll:COREDLL.dll
 0001:00010258       FreeLibrary                10011258 f   coredll:COREDLL.dll
 0001:00010268       GetProcAddressW            10011268 f   coredll:COREDLL.dll
 0001:00010278       DeviceIoControl            10011278 f   coredll:COREDLL.dll
 0001:00010288       LocalFree                  10011288 f   coredll:COREDLL.dll
 0001:00010298       FormatMessageW             10011298 f   coredll:COREDLL.dll
 0001:000102a8       GetLastError               100112a8 f   coredll:COREDLL.dll
 0001:000102b8       CreateFileW                100112b8 f   coredll:COREDLL.dll
 0001:000102c8       CloseHandle                100112c8 f   coredll:COREDLL.dll
 0001:000102d8       OutputDebugStringW         100112d8 f   coredll:COREDLL.dll
 0001:000102e8       DllMain                    100112e8 f   corelib0:dllmain.obj
 0001:00010404       _DllMainCRTStartup         10011404 f   corelib0:pegdmain.obj
 0001:00010434       __GSHandlerCheckCommon     10011434 f   corelib0:gshandler.obj
 0001:00010470       __GSHandlerCheck           10011470 f   corelib0:gshandler.obj
 0001:00010494       __security_init_cookie     10011494 f   corelib0:seccinit.obj
 0001:000104f0       __security_check_cookie    100114f0 f   corelib0:armsecgs.obj
 0001:00010504       __gsfailure                10011504 f   corelib0:armsecgs.obj
 0001:00010610       _cexit                     10011610 f   corelib0:cexit.obj
 0001:0001062c       _initterm                  1001162c f   corelib0:crt0dat.obj
 0001:00010660       _cinit                     10011660 f   corelib0:crt0dat.obj
 0001:00010694       memcpy                     10011694 f   corelib1:COREDLL.dll
 0001:000106a4       swprintf                   100116a4 f   corelib1:COREDLL.dll
 0001:000106b4       calloc                     100116b4 f   corelib1:COREDLL.dll
 0001:000106c4       realloc                    100116c4 f   corelib1:COREDLL.dll
 0001:000106d4       memset                     100116d4 f   corelib1:COREDLL.dll
 0001:000106e4       strlen                     100116e4 f   corelib1:COREDLL.dll
 0001:000106f4       strrchr                    100116f4 f   corelib1:COREDLL.dll
 0001:00010704       strcpy                     10011704 f   corelib1:COREDLL.dll
 0001:00010714       fclose                     10011714 f   corelib1:COREDLL.dll
 0001:00010724       _stricmp                   10011724 f   corelib1:COREDLL.dll
 0001:00010734       atof                       10011734 f   corelib1:COREDLL.dll
 0001:00010744       atoi                       10011744 f   corelib1:COREDLL.dll
 0001:00010754       strstr                     10011754 f   corelib1:COREDLL.dll
 0001:00010764       fgets                      10011764 f   corelib1:COREDLL.dll
 0001:00010774       sprintf                    10011774 f   corelib1:COREDLL.dll
 0001:00010784       fopen                      10011784 f   corelib1:COREDLL.dll
 0001:00010794       malloc                     10011794 f   corelib1:COREDLL.dll
 0001:000107a4       free                       100117a4 f   corelib1:COREDLL.dll
 0001:000107b4       vsprintf                   100117b4 f   corelib1:COREDLL.dll
 0001:000107c4       strncpy                    100117c4 f   corelib1:COREDLL.dll
 0001:000107d4       _vsnprintf                 100117d4 f   corelib1:COREDLL.dll
 0001:000107e4       strcat                     100117e4 f   corelib1:COREDLL.dll
 0001:000107f4       _XcptFilter                100117f4 f   corelib1:COREDLL.dll
 0001:00010804       __C_specific_handler       10011804 f   corelib1:COREDLL.dll
 0001:00010814       __security_gen_cookie2     10011814 f   corelib1:COREDLL.dll
 0001:00010824       __report_gsfailure         10011824 f   corelib1:COREDLL.dll
 0001:00010834       DisableThreadLibraryCalls  10011834 f   coredll:COREDLL.dll
 0001:00010844       TerminateProcess           10011844 f   coredll:COREDLL.dll
 0001:00010898       __IMPORT_DESCRIPTOR_COREDLL 10011898     coredll:COREDLL.dll
 0001:000108ac       __NULL_IMPORT_DESCRIPTOR   100118ac     coredll:COREDLL.dll
 0002:00000000       __imp___GetUserKData       10013000     coredll:COREDLL.dll
 0002:00000004       __imp_CreateEventW         10013004     coredll:COREDLL.dll
 0002:00000008       __imp_WaitForSingleObject  10013008     coredll:COREDLL.dll
 0002:0000000c       __imp_GetTickCount         1001300c     coredll:COREDLL.dll
 0002:00000010       __imp_InterlockedCompareExchange 10013010     coredll:COREDLL.dll
 0002:00000014       __imp_WideCharToMultiByte  10013014     coredll:COREDLL.dll
 0002:00000018       __imp_GetModuleFileNameW   10013018     coredll:COREDLL.dll
 0002:0000001c       __imp_Sleep                1001301c     coredll:COREDLL.dll
 0002:00000020       __imp_LoadLibraryW         10013020     coredll:COREDLL.dll
 0002:00000024       __imp_FreeLibrary          10013024     coredll:COREDLL.dll
 0002:00000028       __imp_GetProcAddressW      10013028     coredll:COREDLL.dll
 0002:0000002c       __imp_DeviceIoControl      1001302c     coredll:COREDLL.dll
 0002:00000030       __imp_LocalFree            10013030     coredll:COREDLL.dll
 0002:00000034       __imp_FormatMessageW       10013034     coredll:COREDLL.dll
 0002:00000038       __imp_GetLastError         10013038     coredll:COREDLL.dll
 0002:0000003c       __imp_CreateFileW          1001303c     coredll:COREDLL.dll
 0002:00000040       __imp_CloseHandle          10013040     coredll:COREDLL.dll
 0002:00000044       __imp_OutputDebugStringW   10013044     coredll:COREDLL.dll
 0002:00000048       __imp_memcpy               10013048     corelib1:COREDLL.dll
 0002:0000004c       __imp_swprintf             1001304c     corelib1:COREDLL.dll
 0002:00000050       __imp_calloc               10013050     corelib1:COREDLL.dll
 0002:00000054       __imp_realloc              10013054     corelib1:COREDLL.dll
 0002:00000058       __imp_memset               10013058     corelib1:COREDLL.dll
 0002:0000005c       __imp_strlen               1001305c     corelib1:COREDLL.dll
 0002:00000060       __imp_strrchr              10013060     corelib1:COREDLL.dll
 0002:00000064       __imp_strcpy               10013064     corelib1:COREDLL.dll
 0002:00000068       __imp_fclose               10013068     corelib1:COREDLL.dll
 0002:0000006c       __imp__stricmp             1001306c     corelib1:COREDLL.dll
 0002:00000070       __imp_atof                 10013070     corelib1:COREDLL.dll
 0002:00000074       __imp_atoi                 10013074     corelib1:COREDLL.dll
 0002:00000078       __imp_strstr               10013078     corelib1:COREDLL.dll
 0002:0000007c       __imp_fgets                1001307c     corelib1:COREDLL.dll
 0002:00000080       __imp_sprintf              10013080     corelib1:COREDLL.dll
 0002:00000084       __imp_fopen                10013084     corelib1:COREDLL.dll
 0002:00000088       __imp___dtos               10013088     corelib1:COREDLL.dll
 0002:0000008c       __imp_malloc               1001308c     corelib1:COREDLL.dll
 0002:00000090       __imp_free                 10013090     corelib1:COREDLL.dll
 0002:00000094       __imp_vsprintf             10013094     corelib1:COREDLL.dll
 0002:00000098       __imp_strncpy              10013098     corelib1:COREDLL.dll
 0002:0000009c       __imp__vsnprintf           1001309c     corelib1:COREDLL.dll
 0002:000000a0       __imp_strcat               100130a0     corelib1:COREDLL.dll
 0002:000000a4       __imp___rt_udiv            100130a4     corelib1:COREDLL.dll
 0002:000000a8       __imp__XcptFilter          100130a8     corelib1:COREDLL.dll
 0002:000000ac       __imp___C_specific_handler 100130ac     corelib1:COREDLL.dll
 0002:000000b0       __imp___security_gen_cookie2 100130b0     corelib1:COREDLL.dll
 0002:000000b4       __imp___report_gsfailure   100130b4     corelib1:COREDLL.dll
 0002:000000b8       __imp_DisableThreadLibraryCalls 100130b8     coredll:COREDLL.dll
 0002:000000bc       __imp_TerminateProcess     100130bc     coredll:COREDLL.dll
 0002:000000c0       \177COREDLL_NULL_THUNK_DATA 100130c0     coredll:COREDLL.dll
 0002:000000cc       gPVRDebugLevel             100130cc     srvclientenvumcmn:pvr_debug.obj
 0002:000000d0       pbtransferqueue_use        100130d0     srvclientsgx:sgxtransfer_context.obj
 0002:000006b0       __security_cookie          100136b0     corelib0:seccinit.obj
 0002:000006b4       __security_cookie_complement 100136b4     corelib0:seccinit.obj
 0002:00000ac1       _exitflag                  10013ac1     corelib0:cexit.obj
 0002:00000ac4       __onexitend                10013ac4     <common>
 0002:00000ac8       __onexitbegin              10013ac8     <common>
 0002:00000acc       _pRawDllMain               10013acc     <common>

 entry point at        0001:00010404

 Static symbols

 0001:00003700       GetApplicationName         10004700 f   pvr_apphint.obj
 0001:00004150       UnmapMemInfoMem            10005150 f   srvclientenvumcmn:pvr_glue.obj
 0001:00004804       CreateDeviceSyncList       10005804 f   srvclientsgx:sgxrender_targets.obj
 0001:0000491c       SetupBackgroundObj         1000591c f   srvclientsgx:sgxrender_targets.obj
 0001:00004a64       SetupRTDataSet             10005a64 f   srvclientsgx:sgxrender_targets.obj
 0001:00005234       FreeRTDataSet              10006234 f   srvclientsgx:sgxrender_targets.obj
 0001:0000595c       CreateSharedPB             1000695c f   srvclientsgx:sgxrender_context.obj
 0001:00005e74       DestroyPerContextPB        10006e74 f   srvclientsgx:sgxrender_context.obj
 0001:00005f94       CreatePerContextPB         10006f94 f   srvclientsgx:sgxrender_context.obj
 0001:00006b44       TQAllocUSEFrag             10007b44 f   srvclientsgx:sgxtransfer_context.obj
 0001:00006e34       TQCreatePDSPrimFrag        10007e34 f   srvclientsgx:sgxtransfer_context.obj
 0001:00006f60       TQCreatePDSSecondaryFrag   10007f60 f   srvclientsgx:sgxtransfer_context.obj
 0001:0000710c       TQCreateHWBGObject         1000810c f   srvclientsgx:sgxtransfer_context.obj
 0001:000071f0       TQCreateFast2DISPControlStream 100081f0 f   srvclientsgx:sgxtransfer_context.obj
 0001:000072c0       TQCreatePixelEventProgram  100082c0 f   srvclientsgx:sgxtransfer_context.obj
 0001:00007ca8       Setup3DRegs                10008ca8 f   srvclientsgx:sgxkick_client.obj
 0001:00007f44       SetupTARegs                10008f44 f   srvclientsgx:sgxkick_client.obj
 0001:0000809c       Update3DRegs               1000909c f   srvclientsgx:sgxkick_client.obj
 0001:00008320       SGXKickSubmit              10009320 f   srvclientsgx:sgxkick_client.obj
 0001:00008bc0       PrepareNormalBlit          10009bc0 f   srvclientsgx:sgxtransfer_queue.obj
 0001:00009fa8       PrepareTextureUpload       1000afa8 f   srvclientsgx:sgxtransfer_queue.obj
 0001:0000a65c       PrepareMipGen              1000b65c f   srvclientsgx:sgxtransfer_queue.obj
 0001:0000ac64       PrepareFillOp              1000bc64 f   srvclientsgx:sgxtransfer_queue.obj
 0001:0000b34c       PrepareBufferBlt           1000c34c f   srvclientsgx:sgxtransfer_queue.obj
 0001:0000b9c4       PrepareCustomOp            1000c9c4 f   srvclientsgx:sgxtransfer_queue.obj
 0001:0000bc58       PrepareFullCustomOp        1000cc58 f   srvclientsgx:sgxtransfer_queue.obj
 0001:0000be7c       PrepareCustomShaderBlit    1000ce7c f   srvclientsgx:sgxtransfer_queue.obj
 0001:0000c5b4       PrepareClipBlit            1000d5b4 f   srvclientsgx:sgxtransfer_queue.obj
 0001:0000cad8       PrepareColourLUTBlit       1000dad8 f   srvclientsgx:sgxtransfer_queue.obj
 0001:0000d190       SGXSubmitTransfer          1000e190 f   srvclientsgx:sgxtransfer_queue.obj
 0001:0000ebd0       SGXTQ_PatchPDSProgram      1000fbd0 f   srvclientsgx:sgxtransfer_utils.obj
 0001:00010308       _DllMainCRTStartupHelper   10011308 f   corelib0:pegdmain.obj
 0001:00010548       doexit                     10011548 f   corelib0:cexit.obj
